:100000000C94EA040C9407050C9407050C9407055E
:100010000C9407050C9407050C9407050C94070530
:100020000C9407050C9407050C9422260C94F426D6
:100030000C944A200C9407050C9407050C940705B2
:100040000C9407050C9407050C9407050C94070500
:100050000C9407050C94D2200C9407050C9407050A
:100060000C9407050C9407050C9407050C940705E0
:100070000C9407050C9407050C9407050C940705D0
:100080000C9407050C9407050C9407050C940705C0
:100090000C9407050C9407050C9407050C940705B0
:1000A0000C9407050C9407050C940705C208C208B8
:1000B000EE08EE08560974098C0A8C0A7F09180AA2
:1000C000290A290A61278827802888278028D42799
:1000D000F72780284E285D2850004F00520051001D
:1000E0005F00600061002E025C005D005E002D007C
:1000F00059005A005B002800620037004F002B00B7
:1001000044454255473A2064697361626C65642EC8
:100110000A0044454255473A20656E61626C656449
:100120002E0A000A0025303258006C65645F746145
:10013000736B3A20004F6E6573686F743A20616389
:10014000746976653A2025640A000A002530386211
:10015000003A200025303258000A722F63203031D7
:100160003233343536370A00290A002575002F004E
:100170002575005D2800256400200025640020000E
:1001800025640020002564007C0025303258006D75
:100190006F7573656B6579205B62746E7C7820790E
:1001A000207620685D287265702F61636C293A2083
:1001B0005B00313A0964656C6179282A31306D73CE
:1001C000293A2025750A323A09696E74657276619A
:1001D0006C286D73293A2025750A333A096D6178C8
:1001E0005F73706565643A2025750A343A0974694D
:1001F0006D655F746F5F6D61783A2025750A353AD9
:1002000009776865656C5F6D61785F7370656564BB
:100210003A2025750A363A09776865656C5F746916
:100220006D655F746F5F6D61783A2025750A0070A7
:100230003A097072696E742076616C7565730A6430
:100240003A097365742064656661756C74730A7528
:10025000703A092B310A646E3A092D310A6C743AEE
:10026000092B31300A72743A092D31300A45534353
:100270002F713A09717569740A0A73706565642093
:100280003D2064656C7461202A206D61785F737015
:10029000656564202A2028726570656174202F20AE
:1002A00074696D655F746F5F6D6178290A77686541
:1002B00072652064656C74613A20637572736F7245
:1002C0003D25642C20776865656C3D25640A53657F
:1002D0006520687474703A2F2F656E2E77696B698C
:1002E00070656469612E6F72672F77696B692F4D36
:1002F0006F7573655F6B6579730A004D3E20004D25
:1003000025753A25733E20003F0A003D2025750AD9
:10031000003F0A0064656661756C74730A00257598
:100320000A003F0A000A092D2056616C756573208A
:100330002D0A00710A000A092D204D6F7573656B37
:100340006579202D0A003F00433E20004C25640AB9
:10035000000A092D20537461747573202D0A686F8B
:1003600073745F6B6579626F6172645F6C656473EF
:1003700028293A20253032580A6B6579626F6172FC
:10038000645F70726F746F636F6C3A2025303258FF
:100390000A6B6579626F6172645F69646C653A20AB
:1003A000253032580A74696D65725F726561643315
:1003B0003228293A202530386C580A000A092D20A5
:1003C00056657273696F6E202D0A5649443A203083
:1003D000784242383028486578776972652920501C
:1003E00049443A20307830353034284E756D70618C
:1003F0006420323029205645523A2030783030304F
:10040000310A4255494C443A202028466562203240
:10041000372032303232290A4F5054494F4E533A26
:10042000204C554641204D4F5553454B455920458D
:10043000585452414B455920434F4E534F4C452041
:10044000434F4D4D414E44203531320A4743433AE4
:1004500020352E342E30204156522D4C4942433AFD
:1004600020322E302E30204156525F415243483ABE
:1004700020617672350A000A092D20436F6E736F72
:100480006C65202D0A4553432F713A0971756974C3
:100490000A6D3A096D6F7573656B65790A000A0913
:1004A0002D204D61676963202D0A443A0944656235
:1004B0007567204D65737361676520546F67676C5E
:1004C000650A583A094D617472697820446562750D
:1004D00067204D6F646520546F67676C65202D2021
:1004E00053686F77206B65797072657373657320DD
:1004F000696E206D617472697820677269640A4B55
:100500003A094B6579626F61726420446562756770
:1005100020546F67676C65202D2053686F77206BC0
:1005200065797072657373207265706F72740A4DAD
:100530003A094465627567204D6F75736520546F85
:1005400067676C650A563A0956657273696F6E0A79
:10055000533A095374617475730A433A09416374D9
:10056000697661746520436F6E736F6C65204D6FA3
:1005700064650A46312D4631303A09537769746310
:100580006820746F204C6179657220302D392028E5
:10059000463130203D204C30290A302D393A09535C
:1005A000776974636820746F204C617965722030BC
:1005B0002D390A47524156453A09537769746368A1
:1005C00020746F204C6179657220302028616C7432
:1005D00065726E617465290A423A094A756D702028
:1005E000746F20426F6F746C6F616465720A45535B
:1005F000433A094A756D7020746F20426F6F746CB6
:100600006F616465722028616C7465726E617465D7
:10061000290A453A095072696E7420454550524F77
:100620004D2053657474696E67730A425350414399
:10063000453A09436C65617220454550524F4D0A59
:10064000006B65796D61705F636F6E6669672E72AE
:1006500061773A20253032580A2E737761705F63D4
:100660006F6E74726F6C5F636170736C6F636B3A03
:100670002025750A2E636170736C6F636B5F746FF6
:100680005F636F6E74726F6C3A2025750A2E7377F4
:1006900061705F6C63746C5F6C6775693A20257577
:1006A0000A2E737761705F7263746C5F726775692D
:1006B0003A2025750A2E737761705F6C616C745FE8
:1006C0006C6775693A2025750A2E737761705F72C1
:1006D000616C745F726775693A2025750A2E6E6FBA
:1006E0005F6775693A2025750A2E737761705F67B9
:1006F000726176655F6573633A2025750A2E73779C
:1007000061705F6261636B736C6173685F62616388
:100710006B73706163653A2025750A2E6E6B726F7C
:100720003A2025750A0064656275675F636F6E66BF
:1007300069672E7261773A20253032580A2E656E2D
:1007400061626C653A2025750A2E6D617472697854
:100750003A2025750A2E6B6579626F6172643A20C2
:1007600025750A2E6D6F7573653A2025750A00652B
:1007700065636F6E6669673A0A64656661756C7475
:100780005F6C617965723A2025750A003F000A6D39
:100790006F7573653A206F66660A000A6D6F757330
:1007A000653A206F6E0A000A6B6579626F61726448
:1007B0003A206F66660A000A6B6579626F6172643F
:1007C0003A206F6E0A000A6D61747269783A206F80
:1007D00066660A000A6D61747269783A206F6E0A63
:1007E000000A64656275673A206F66660A000A64EB
:1007F000656275673A206F6E0A000A0A4A756D7065
:10080000696E6720746F20626F6F746C6F616465CE
:10081000722E2E2E2000433E2000436C65617269CB
:100820006E6720454550524F4D0A000A0025303270
:100830005820006B6579626F6172645F7265706FDA
:1008400072743A20005B735D005B575D005B535D23
:10085000005B525D005B445D005B435D0014034E32
:100860000075006D007000610064002000320030EF
:1008700000000010034800650078007700690072EE
:1008800000650000000403090409025B0003010085
:10089000A0FA09040000010301010009211101006F
:1008A000012240000705810308000109040100013D
:1008B00003000000092111010001227B00070582CD
:1008C00003200001090402000203000000092111B5
:1008D0000100012222000705830320000107050310
:1008E00003200001120100020000000880BB040583
:1008F0000100010200010631FF0974A1010975150B
:100900000026FF009520750881020976150026FF54
:1009100000952075089102C005010902A101850218
:100920000901A100050919012908150025019508EB
:10093000750181020501093009311581257F950274
:100940007508810609381581257F9501750881068E
:10095000050C0A38021581257F950175088106C0AE
:10096000C005010980A101850319012AB7001501FD
:1009700026B700950175108100C0050C0901A10181
:10098000850419012AA002150126A00295017510FF
:100990008100C005010906A101050719E029E71535
:1009A00000250195087501810295017508810105F1
:1009B00007190029FF150026FF009506750881001C
:1009C0000508190129059505750191029501750321
:1009D0009101C00011241FBECFEFDAE0DEBFCDBF12
:1009E00011E0A0E0B1E0ECE7F2E502C005900D9265
:1009F000A03FB107D9F722E0A0EFB1E001C01D92FE
:100A0000A43BB207E1F70E94A2160C943C290C9477
:100A10000000FF93EF93E091F001F091F101309726
:100A200009F00995EF91FF910895FC0185918030BF
:100A300011F0EFDFFBCF0895FF27E0E230E247FF40
:100A40000CC0419597FF09C0EDE2609570958095C7
:100A50009095611D711D811D911D27FF02C021957B
:100A600030E350E2AA27660F771F881F991FAA1F3D
:100A7000A41710F0A41B63955A95A9F7AA3008F0A3
:100A8000A95FA05DAF93F39561157105810591058F
:100A900041F7ED3211F4EF93F395F21718F43F9309
:100AA000F395FBCF8F91B5DFFA95E1F70895E991C2
:100AB000F9918591803021F0853219F0AADFF9CFC4
:100AC000089520E0E89455915532C1F3503311F464
:100AD000689455915A3348F4505390F3220F022EE4
:100AE000220F220F200D250FF4CF0EF421958991AE
:100AF0009991533619F3533729F1533559F1BC0104
:100B000088279927E8945C3621F489919991689413
:100B10005591543639F446EF7EF077FF0DC08FEFD4
:100B20009FEF0AC055374AE039F0583540E121F0CF
:100B3000523642E009F00895FF93EF937DDFEF9185
:100B4000FF91B7CFFF93EF93FC0181918030B9F310
:100B500060DFFBCFFF93EF9368DFF1CFDF93CF939D
:100B6000CDB7DEB72596A3DFCF91DF91089581E061
:100B7000089581E008950C94B90508950C94BD057D
:100B80001F93CF93DF9300D000D01F92CDB7DEB775
:100B900049835A836B833091F30189819A813111A2
:100BA00014C0662359F0222349F00E94C70C182F65
:100BB000682F89819A810E94720C03C00E949C0C4C
:100BC000182F69817A81812F04C00E94C70C698126
:100BD0007A810F900F900F900F900F90DF91CF912F
:100BE0001F910C94F613FC01262F408151816281E4
:100BF000738184810C94C00581E00895CF93DF93C5
:100C0000EC0160E00E94F305BE01DF91CF910C94EE
:100C1000BE050C9466150C94621508950E941C0B79
:100C20000E940D062FEF84E39CE02150804090400D
:100C3000E1F700C000000C94F8200F931F93CF93AE
:100C4000DF938C0161E00E94F305EC01B8010E9482
:100C5000BB05882309F45BC0B801CE010E94D81EF1
:100C6000882309F454C0B801CE010E94BA19882320
:100C700009F44DC0B801CE010E94341E882309F446
:100C800046C0F80182818823D9F1CF3D8CE5D80791
:100C900079F140F4C115FCE5DF0791F0C130DC4586
:100CA00091F02EC0CC35EDE5DE0741F1CD35FDE507
:100CB000DF0709F1CB35DD4519F50E945E1120C033
:100CC0000E940E0624C080916402C82FC095C17096
:100CD000C0FB80F980936402CC2329F082E191E08B
:100CE0000E94150514C080E091E00E94150510C017
:100CF0000E940C120CC00E94551102C00E9461118A
:100D0000C801DF91CF911F910F910C94B705C0E0FE
:100D10008C2FDF91CF911F910F9108950E942D206C
:100D20000C94B9060E94BC060C9433208295982F2F
:100D3000937344E0949F900111248C7C8695869552
:100D4000282B822F8575880F2A7A2695822B089565
:100D500008950C94A80681E008950C94AB060895BC
:100D6000CF93C82F0E94A9068C2F0E94AD06CF9169
:100D7000089580E00C94B0060E94341F0C94B006D5
:100D8000CF930E94341FC82F8091F201C81741F100
:100D9000C093F2018091640282FF1EC080FF04C0F4
:100DA0008AE291E00E9415058091640280FF0CC0E8
:100DB0001F92CF9385E291E09F938F930E94AE059F
:100DC0000F900F900F900F908091640280FF04C0ED
:100DD00083E291E00E9415058C2FCF910C94B00610
:100DE000CF910895CF93DF93CDB7DEB72B970FB692
:100DF000F894DEBF0FBECDBF4F83588769877A87CF
:100E00008B8761110E948D109E012F5F3F4F86E0FE
:100E1000F90111928A95E9F785E0FE013796D9012B
:100E200001900D928A95E1F789819A814C815D81CB
:100E3000452B31F09F3F31F491E08F3F19F403C00F
:100E400091E001C090E090FF09C049815A816B8117
:100E50007C818D819E810E94AE0F05C0C9010E94D8
:100E6000FC058111F2CF2B960FB6F894DEBF0FBEB2
:100E7000CDBFDF91CF910895FC01808191810E94C7
:100E8000090D0895CF93882309F4A9C0C82F82388B
:100E9000C1F40E94341F81FDA2C069E38091020168
:100EA000909103010E9405200E94AF102FEF81EE68
:100EB00094E0215080409040E1F700C0000069E3D9
:100EC00019C0833801F50E94341F80FD88C063E596
:100ED00080910201909103010E9405200E94AF10B1
:100EE0002FEF81EE94E0215080409040E1F700C068
:100EF000000063E580910201909103010E940720A8
:100F0000CF910C94AF108438C1F40E94341F82FD3D
:100F100066C067E480910201909103010E94052060
:100F20000E94AF102FEF81EE94E02150804090405E
:100F3000E1F700C0000067E4DDCF8CEF8C0F813A51
:100F4000F8F48C2F0E94DD1D811149C06C2F809117
:100F50000201909103010E94CF1F882349F06C2F5A
:100F600080910201909103010E9407200E94AF101E
:100F70006C2F80910201909103010E940520C0CF47
:100F800080E28C0F883048F4C77081E001C0880F80
:100F9000CA95EAF70E947010B3CFEBE5EC0FE3308F
:100FA00040F4F0E0E95BFE4F808190E0CF910C943B
:100FB000971FE8E5EC0FE73150F4F0E0EE0FFF1F6C
:100FC000E75EFE4F80819181CF910C94AD1FCD3EA5
:100FD00030F08C2F0E942717CF910C94F917CF91E6
:100FE0000895882309F464C0823879F40E94341F7C
:100FF00081FF5EC069E380910201909103010E942C
:1010000005200E94AF1069E310C08338B1F40E943C
:10101000341F80FF4DC063E5809102019091030170
:101020000E9405200E94AF1063E58091020190911B
:1010300003010E9407200C94AF10843879F40E94B9
:10104000341F82FF35C067E4809102019091030153
:101050000E9405200E94AF1067E4E7CF9CEF980F35
:10106000913A10F4682FE1CF90E2980F983050F445
:10107000877091E001C0990F8A95EAF7892F0E9445
:101080007610D9CF9BE5980F933020F480E090E064
:101090000C94971F98E5980F973120F480E090E02A
:1010A0000C94AD1F8D3E20F00E9482170C94F9170E
:1010B00008951F93CF93DF93182FEB010E944207EF
:1010C000209741F08FE99FE00197F1F700C0000001
:1010D0002197F6CF812FDF91CF911F910C94F107CB
:1010E000893319F060E070E002C060E570E00C94B4
:1010F0005908882321F00E9470100C94AF100895B5
:10110000882321F00E9476100C94AF100895CF929E
:10111000DF92EF92FF920F931F93CF93DF937C01A7
:10112000D62FC72FFC011281058102950F700E94F6
:1011300066108823B9F01123A9F08C2F807F8034AA
:1011400021F080E28D0F883068F08091980282FD56
:1011500009C082E00E940F110E94661091E0D82E13
:10116000D92601C0D12CCC2EC2948FE0C8228C2D60
:1011700090E08C30910508F0CFC1FC01EA5AFF4F96
:101180000C94D3288C2F807FCF70882311F0C295C8
:10119000C07F112399F0CC2309F4AAC180E28D0FFE
:1011A000883010F0D11104C08C2F0E94701003C041
:1011B0008C2F0E9480100E94AF109AC18D2F0E9428
:1011C000F107CC2309F4A8C180E28D0F883038F1F3
:1011D000DD2329F18C2F0E94861024C08C2F807F64
:1011E000CF70803211F0C295C07FDD2319F0D1306D
:1011F000A1F13DC08091980282FF17C0112349F0F0
:10120000CC2329F08C2F0E9470100E94AF1080E038
:1012100070C180E00E94F107CC2309F47DC18C2FBE
:101220000E9476100E94AF1077C1112371F0002345
:1012300041F0013031F40E9490108C2B0E949810E4
:101240006BC10E9490108C2B1DC0002319F001303F
:1012500009F462C10E94A51025C0112321F00630B7
:1012600008F05AC10EC0053008F056C11BC011234A
:1012700061F0002331F0F701858180FF39C18F7063
:1012800085838C2F0E94790847C1002359F0D933F8
:1012900009F03FC1FFEF07EE13E0F15000401040AE
:1012A000E1F735C18C2F0E94800836C18C2F8695BE
:1012B0008695837019F0813061F02EC1112321F0E1
:1012C0008D2F9C2F937002C080E090E00E94971FAA
:1012D0002BC1112321F08D2F9C2F937002C080E031
:1012E00090E00E94AD1F20C18D2F112319F00E94A4
:1012F000271702C00E9482170E94F91715C18C2F70
:10130000837009F047C011110BC12D2F229526952E
:101310002770220F220F6D2F6F70862F90E0A0E0B4
:10132000B0E0022E04C0880F991FAA1FBB1F0A94A9
:10133000D2F7D4FF10C04FE050E060E070E004C08E
:10134000440F551F661F771F2A95D2F74095509579
:101350006095709503C040E050E0BA01C695C6950F
:10136000C3708A019B01082B192B2A2B3B2BC90127
:10137000B801C23049F058F4C13019F00E94880B0E
:10138000CFC00E94760BCCC00E949A0BC9C00E94AD
:10139000740BC6C0112319F08C2F817001C0869583
:1013A000882309F4BDC02D2F229526952770220F82
:1013B000220F6D2F6F70862F90E0A0E0B0E0022E1C
:1013C00004C0880F991FAA1FBB1F0A94D2F7D4FF2D
:1013D00010C04FE050E060E070E004C0440F551FC3
:1013E000661F771F2A95D2F74095509560957095A6
:1013F00003C040E050E0BA01C695C695C3708A01AB
:101400009B01082B192B2A2B3B2BC901B801C23099
:1014100049F058F4C13019F00E944D0C81C00E946F
:101420003B0C7EC00E945F0C7BC00E94AE0B78C05C
:10143000CF70112339F08C2F0E94D40B8D2F0E9476
:1014400079086EC08D2F0E9480088C2F0E94F50BAA
:1014500067C0D23F21F128F4D03F41F0D13FC1F025
:1014600043C0D33F19F1D43F79F03EC0112341F07E
:10147000053008F051C08C2F8F710E941A0C4CC09F
:10148000063008F049C0F7CF8091980282FF18C05B
:10149000112339F08C2F8F710E94D40B3DC0112382
:1014A000C9F38C2F8F710E94F50B36C0112329F0E0
:1014B0008C2F8F710E94BF0B2FC00E94BA0B2CC0C3
:1014C000112349F0CF718C2F0E94D40B63E08C2F35
:1014D0000E94F41021C081E00E940F110230E0F060
:1014E00082E00E940F1118C0112331F0002391F205
:1014F0008D2F0E94420710C0002399F2D93349F47E
:101500001FEF27EE33E0115020403040E1F700C0DC
:1015100000008D2F0E94F10788EF8C0D843020F49D
:101520000E94341F0E94B006DD20C9F00E946210A4
:1015300080FD15C0F70112820E945C100E94D40B3E
:10154000C7010E94D00A0E945C10DF91CF911F91C9
:101550000F91FF90EF90DF90CF900C94F50BDF91FF
:10156000CF911F910F91FF90EF90DF90CF90089552
:101570000F931F93CF93DF93EC01688179818A8168
:101580000E94140D8C010E94710C0E94620BB80124
:10159000CE010E948708DF91CF911F910F9108958E
:1015A000CF93DF93EC01988189812B813C81232BA0
:1015B00031F08F3F31F481E09F3F19F403C081E0A7
:1015C00001C080E080FD1DC0CE010E941D0681117A
:1015D00010C00E9466108823A1F08A81882389F0B8
:1015E0008091980282FD0DC082E0DF91CF910C9432
:1015F0000F11CE010E94B80ACE01DF91CF910C9459
:10160000FE05DF91CF91089580E090E00E94971F42
:1016100080E090E00E94AD1F0E948D100E94AF10EC
:101620000E94AC190C94F91780910201909103016A
:101630000E9409200C94040B0E947D100C94140B42
:1016400092959F70963079F010F4925001C09A50A4
:10165000923068F4803F69F018F4883E40F409C085
:10166000843F29F406C0883E20F0813F11F080E0DD
:10167000089581E00895FC01808191810E94090D07
:101680000E94200B0895CF93DF9300D000D01F92CB
:10169000CDB7DEB70F900F900F900F900F90DF91A6
:1016A000CF910895CF93DF9300D000D000D0CDB775
:1016B000DEB726960FB6F894DEBF0FBECDBFDF9122
:1016C000CF910895089508950C94630B0C94640BC6
:1016D0000E94660B609307027093080280930902D0
:1016E00090930A020C94040B0C94680B0F931F93B5
:1016F00000910702109108022091090230910A021C
:10170000602B712B822B932B1F910F910C94680BE4
:101710000F931F9300910702109108022091090274
:1017200030910A0260237123822393231F910F912A
:101730000C94680B0F931F930091070210910802FD
:101740002091090230910A0260277127822793278E
:101750001F910F910C94680B0C94630B0E94AC0BBF
:101760006093030270930402809305029093060233
:101770000C94040B60E070E0CB010C94AE0B0F9363
:101780001F9341E050E060E070E08A019B0104C0DB
:10179000000F111F221F331F8A95D2F7C901B8010C
:1017A0001F910F910C94AE0B0F931F9341E050E0EB
:1017B00060E070E004C0440F551F661F771F8A95D4
:1017C000D2F78091030290910402A0910502B0919A
:1017D00006028A019B01082B192B2A2B3B2BC901DE
:1017E000B8011F910F910C94AE0B0F931F9341E022
:1017F00050E060E070E004C0440F551F661F771F83
:101800008A95D2F740955095609570958091030226
:1018100090910402A0910502B09106028A019B01F9
:10182000082319232A233B23C901B8011F910F91D3
:101830000C94AE0B0F931F9341E050E060E070E01A
:1018400004C0440F551F661F771F8A95D2F78091F9
:10185000030290910402A0910502B09106028A0150
:101860009B01082719272A273B27C901B8011F9187
:101870000F910C94AE0B0F931F93009103021091E4
:1018800004022091050230910602602B712B822BFD
:10189000932B1F910F910C94AE0B0F931F930091FC
:1018A0000302109104022091050230910602602388
:1018B0007123822393231F910F910C94AE0B0F93EE
:1018C0001F930091030210910402209105023091B0
:1018D000060260277127822793271F910F910C948E
:1018E000AE0B0895990F990F890FE82FE695E695AD
:1018F000E695877051E001C0550F8A95EAF785E0BB
:10190000E89FF0011124EC50FE4F20E030E070E041
:101910004081CB01022E02C0969587950A94E2F78A
:101920008170819584278523842781932F5F3F4F82
:101930002530310569F70895990F990F890F682FA0
:10194000669566956695982F977085E0689FB001BB
:10195000112440E050E080E0FB01E40FF51FEC5063
:10196000FE4F208130E0092E02C0369527950A945B
:10197000E2F721703327042E01C0220F0A94EAF700
:10198000822B4F5F5F4F4530510531F70895BF926D
:10199000CF92DF92EF92FF920F931F93CF93DF933B
:1019A0008C01C0900302D0900402E0900502F090F8
:1019B00006028091070290910802A0910902B0915D
:1019C0000A02C82AD92AEA2AFB2ACFE1D0E0D701A5
:1019D000C6010C2E04C0B695A795979587950A94D5
:1019E000D2F780FD04C0219790F7B12C07C0BC2E20
:1019F000B8018C2F0E940A140197A9F38B2DDF9157
:101A0000CF911F910F91FF90EF90DF90CF90BF90FB
:101A10000895CF93DF93EC010E94C70CBE010E9492
:101A20000A14DF91CF9108951F93CF93DF93EB01B9
:101A30009091F301992321F0CB010E94090D13C06D
:101A4000882349F0CB010E94C70C182F682FCE01C4
:101A50000E94720C04C0CB010E949C0C182FBE0186
:101A6000812F0E940A14DF91CF911F9108951F9337
:101A7000CF93DF93C0910B0216E080910C02C81740
:101A800099F0D0E01C9FF0011D9FF00D1124E35F41
:101A9000FD4F4081518162817381848195810E94D3
:101AA000520B2196C770E9CFDF91CF911F91089516
:101AB00040913D0250913E0260913F027091400280
:101AC00080914102909142020C94520BEF92FF924E
:101AD0000F931F93CF93DF938091420282958F7073
:101AE00009F065C080913F02882309F460C08091AD
:101AF0000B02F0900C0210913D0200913E026091A9
:101B000040027091410291E01F3F09F090E0C091C6
:101B10000001D0910101292F96E0E92E8F1509F4DB
:101B200046C06115710521F00F3F21F030E003C080
:101B300031E001C0322F90E030FD36C0E89EF00168
:101B4000E99EF00D1124DF01A35FBD4F11963C917A
:101B50001197301329C03C91311326C012963C9145
:101B60001297311121C013964D915C911497461B29
:101B7000570B4C175D07C0F4809142028F70806153
:101B800080934202EE5EFD4F80818F708061808382
:101B90008DE392E00E94D00ADF91CF911F910F91C7
:101BA000FF90EF900C94370D01968770B7CFDF91BF
:101BB000CF911F910F91FF90EF9008959F92AF9258
:101BC000BF92CF92DF92EF92FF920F931F93CF932A
:101BD000DF93CDB7DEB761970FB6F894DEBF0FBEC7
:101BE000CDBF8C0185E0F801DE011D9601900D92BC
:101BF0008A95E1F7D8011296EC9090913D02E09120
:101C00003E0220914002309141022115310531F010
:101C1000EF3F31F481E09F3F19F403C081E001C040
:101C200080E0B82FB1709B2E80FD47C1D8014C9148
:101C300011965C9111971396AD90BC9014978DE31B
:101C4000C82E82E0D82EF0903F02B501621B730BC4
:101C50002091000130910101FF2009F4D9C0809149
:101C600042026217730708F095C0282F207F09F001
:101C700052C05E1313C0491311C0FE2CE1100EC0F8
:101C80008F708061809342020E94580DC6010E94AD
:101C9000D00A80914202F80185834DC1AB2831F012
:101CA0005F3F31F481E04F3F19F403C081E001C090
:101CB00080E080FD03C081E08E2502C080E090E0DE
:101CC000F82FF170FF2E80FF1CC080910B02209135
:101CD0000C0236E0821709F40BC190E0389FF00146
:101CE000399FF00D1124E35FFD4F6181561306C04B
:101CF0006081461303C06281E61203C001968770BB
:101D0000E9CFFE2CEE2009F416C1809142028160D9
:101D10008093420254C05E1306C0491304C0E11010
:101D200002C0F80199C0C8010E943B0B882361F1F1
:101D3000EE2051F120914202822F82958F7090E027
:101D4000029774F080913D0290913E0298878F83B4
:101D50001986BB86AA862C87CE0107960E94D00AD8
:101D600086E0F801ADE3B2E001900D928A95E1F7CB
:101D70000E94660D0E94580D0AC05E1711F1C8013D
:101D80000E943B0B81112CC0C8010E94D00AFF2485
:101D9000F394D1C0282F207F81F77A2DB98AA88AA1
:101DA0006E2D89890E94430B8DE392E00E94D00A38
:101DB00086E0D6011D928A95E9F70E94580DF12C14
:101DC000BAC04913DCCFE110DACFF8018583C8012E
:101DD0000E94D00A86E0D6011D928A95E9F7ABC031
:101DE000EE2091F220914202822F82958F7090E036
:101DF00002970CF4B5CF80913D0290913E029A83F8
:101E000089831B82BD82AC822E83CE010196A6CF30
:101E10006217730708F044C0FE2CEE2009F4B4CF1B
:101E20005E1330C049132EC02091420220FD21C014
:101E3000822F82958F70482F50E041155105C9F0CF
:101E4000F80125834F30510541F08F5F982F92950F
:101E5000907F822F8F70892B8583C8010E94D00AC2
:101E600086E0F801ADE3B2E001900D928A95E1F7CA
:101E70003CC086E0F801ADE3B2E001900D928A9596
:101E8000E1F759C0C8010E943B0B811169CF8091D5
:101E90004202816080934202C8010E94D00A4BC076
:101EA0007A2DB98AA88A6E2D89890E94430B86E013
:101EB000D6011D928A95E9F718C0EE2009F464CF87
:101EC000C8010E943B0BF82E882309F45DCF86E001
:101ED000F801ADE3B2E001900D928A95E1F78DE350
:101EE00092E00E943C070E94660D0E94580D23C09C
:101EF0004D875E878D859E850E94090D292F22952D
:101F00002F70223028F49F7039F0811105C00BC06A
:101F1000243028F49F7049F4805E883020F0C80196
:101F20000E94D00A9F2CF92C06C0D80115969C91CE
:101F3000907F91F7F8CF8F2D61960FB6F894DEBFA2
:101F40000FBECDBFDF91CF911F910F91FF90EF900A
:101F5000DF90CF90BF90AF909F9008951F93CF9345
:101F6000DF93CDB7DEB72C970FB6F894DEBF0FBE68
:101F7000CDBF4F83588769877A878B879C87CE012F
:101F800007960E94DE0D8823D1F09F8188852A85DF
:101F90003B85232B31F08F3F31F481E09F3F19F4D3
:101FA00003C081E001C080E080FD47C04F815885BB
:101FB00069857A858B859C850E94520B3EC086E0A0
:101FC000FE013796DE01119601900D928A95E1F798
:101FD000FF81E8856A857B856115710531F0EF3FEA
:101FE00031F481E0FF3F19F403C081E001C080E0DB
:101FF00080FD23C020910C0230E0C901019687705A
:10200000992740910B0250E084179507F1F1F9836D
:10201000EA837D836C8396E0929FD001939FB00DFD
:102020001124A35FBD4FFE01319601900D929A9548
:10203000E1F780930C020E94370D16E080910B02AD
:1020400090910C02891771F1189FC0011124835FD0
:102050009D4F0E94DE0D882329F1E0910B021E9F07
:10206000F0011124E35FFD4F408151816281738152
:10207000848195810E94520B80910B0290E0019621
:102080008770992780930B02D9CF0E941C0B109266
:102090000C0210920B02EDE3F2E086E0DF011D92EC
:1020A0008A95E9F72C960FB6F894DEBF0FBECDBF28
:1020B000DF91CF911F91089580914B028595859571
:1020C0008595089580914B028770089590914B02F9
:1020D000977081E009F480E0089580915602089598
:1020E00090915602892B8093560208958095909185
:1020F000560289238093560208951092560208953D
:1021000090915502892B8093550208958095909166
:10211000550289238093550208951092550208951F
:1021200080914C02089508950C9493100C9494108F
:102130009091980292FD08C090914C02981721F05E
:1021400080934C020C949610089580914C02882341
:1021500029F010924C0280E00C9496100895CF93D1
:10216000DF93E0910201F091030180915602808398
:10217000E0910201F0910301908180915502892B39
:10218000808380914C02882381F0E0910201F091DC
:1021900003019081892B808380910201909103013A
:1021A0000E94C31F81110E94A510C0910201D0910D
:1021B000030148E050E063E472E0CE010E94ED28A4
:1021C000892B69F088E0FE01A3E4B2E001900D9252
:1021D0008A95E1F7CE01DF91CF910C94401FDF91FA
:1021E000CF9108950C9493109091980292FD10C095
:1021F00098E0899F90011124262B20934B020E9486
:10220000D40B80914B028595859585950C94F210A1
:102210000C94D40B10924B0280E00C94F21020919D
:102220004B028095822380934B02982F977099F4EC
:1022300030E0482F082E000C550B2417350759F0B5
:102240009091980292FD07C08595859585950E948D
:10225000F50B0C940A110895CF939091980292FB7C
:10226000222720F92817F9F0C82F892FC0FB82F9FF
:102270008093980280919702909198020E94881111
:1022800082E00E940F118091640280FF0CC01F92B7
:10229000CF9385E391E09F938F930E94AE050F90BB
:1022A0000F900F900F90CF9108958091980282FB2C
:1022B000882780F991E089270C942C1181E00C94F7
:1022C0002C1180E00C942C1180E090E00E940229F7
:1022D00021E0893E9E4F09F020E0822F089582E0A0
:1022E00090E00C94FA2883E090E00C94FA28CF93C5
:1022F00084E090E00E94FA28C82F82E290E00E94D9
:10230000FA282C2F30E0A901582BCA01CF9108954B
:10231000CF93C92F682F84E090E00E9408296C2F8A
:1023200082E290E0CF910C940829AB01BC018FE0D0
:1023300090E00C941A29AB01BC0183E190E00C946D
:102340001A2960E070E0CB010C949B1160E070E012
:10235000CB010E9495110C94A11169EE7EEF80E0F3
:1023600090E00E94262960E082E090E00E94082927
:1023700060E083E090E00E9408291092070210922A
:1023800008021092090210920A0260E084E090E0D4
:102390000E94082960E082E290E00E94082960E043
:1023A00085E090E00E94082960E086E090E00E94CD
:1023B00008296FEF87E090E00E94082940E050E094
:1023C000BA0188E090E00E941A2960E08DE090E078
:1023D0000E94082940E050E0BA0188E190E00E94A4
:1023E0001A2960E087E190E00E94082940E050E06F
:1023F000BA018CE190E00E941A2960E070E080E26E
:1024000090E00E94262940E050E0BA0188E190E087
:102410000E941A290C94A6110C94AD11682F8EE01D
:1024200090E00C9408290E94B7206093600270939A
:102430006102809362029093630260935C027093E6
:102440005D0280935E0290935F02089585B7806875
:1024500085BF85B7806885BF089581E008950C9495
:102460002D1208950C9431120C9431120C943412E4
:102470000C9431120C9438120C9431120E942612D2
:102480008DEF92E20E942A1F0E943C120C943A1295
:102490000E9432120C9431120E94E7140C94AF0681
:1024A0000E94A2200E9403160E944C120C94361225
:1024B0008F929F92AF92BF92CF92DF92EF92FF9254
:1024C0000F931F93CF93DF93CDB7DEB72A970FB645
:1024D000F894DEBF0FBECDBF0E941816982E811152
:1024E0000E94131287E5A82E82E0B82E00E010E0CB
:1024F000802E802F0E940B15D82EF501C1905F0110
:10250000C826B1F40F5F1F4F0530110589F78FEF13
:1025100089838A831B820E94AB208160782F9D83F0
:102520008C8349815A816B818D810E94F2062FC074
:102530008091640281FD0E941115E12CFF24F39427
:102540008C2D8F21F1F00E942F12882399F0EE82BA
:102550008F82DF2081E009F480E088870E94AB2031
:102560008160782F9A8789874E815F8168858A8507
:102570000E94F206F801E95AFD4F8081F826F082A8
:1025800006C0E394FF0CF4E0EF12DACFBBCF81E09A
:10259000911001C080E02A960FB6F894DEBF0FBEFE
:1025A000CDBFDF91CF911F910F91FF90EF90DF9002
:1025B000CF90BF90AF909F908F9008950E94581237
:1025C0000E9499180C94C006CF93DF930E940F14B9
:1025D000EC01811521E5920708F045C0811530E531
:1025E000930708F094C0883E910528F5803E910538
:1025F00008F0F8C0883A910570F4853A910508F022
:102600007CC08130910509F475C008F4E8C00497D6
:1026100008F0E8C0E4C08F3B910508F0E0C0C85A5C
:10262000D0E0CC0FDD1FC65BDE4F0990D881C02DF6
:10263000CE019464D8C0811540E2940758F4811506
:1026400051E0950708F0CEC08D3E910508F4C7C053
:102650009065C9C0C11580E4D80708F4C0C0DF7018
:10266000CE01906AC0C0811525E59207A8F48115B6
:1026700034E5930708F095C0811543E5940708F009
:102680007BC0811552E5950708F061C0D82FCC2793
:10269000CE01816F906AA7C0C11589E5D807A0F463
:1026A000C11528E5D20708F082C0C11536E5D30769
:1026B00008F095C08C2F0E94A3148F7190E0D82F42
:1026C000CC27CE0190628FC0C1154AE5D40708F42B
:1026D00074C0CE0190568115904208F080C08D2FB5
:1026E0008F710E94A314DD27D0628F71AE01582B29
:1026F000CA0179C081E090E076C0C55AD0E0C858E0
:10270000DE4F8881C82FD0E0CE0190646CC074E0A9
:10271000969587957A95E1F7282F23703C2F337093
:1027200081E090E002C0880F991F3A95E2F79C681B
:10273000AC01522B9A019C2F9F709695969550E272
:10274000959FE0011124C9018C2B9D2B4CC08370F7
:10275000992721E030E002C0220F331F8A95E2F76B
:102760009C2F9695969580E2989FE0011124C22BAC
:10277000D32BCE019C6837C08370992721E030E0CD
:1027800002C0220F331F8A95E2F79C2F96959695EB
:1027900040E2949FE0011124C22BD32BCE019A6812
:1027A00022C0D82FCC27CE01846F906A1CC0DC2FAA
:1027B000CC27CE01806F906A16C08C2F8F700E943C
:1027C000A31494E0D695C7959A95E1F7CF70D0E021
:1027D000DC2FCC27D0699E01282BC90104C080E0E2
:1027E00090E001C0CE01DF91CF910895E72FF0E096
:1027F00095E0899FE00DF11D1124EE0FFF1FEE0FF4
:10280000FF1FE60FF11DEE0FFF1FE852FF4F8591EE
:10281000949108950E94F6130E94E412089582385C
:10282000910569F1B0F48133910509F46DC048F464
:102830008932910509F463C08A32910509F469C0AF
:1028400008958533910509F455C089339105B9F090
:102850000895833E910569F138F4803E9105B1F009
:10286000823E910509F10895863E9105A9F1873EC2
:102870009105B9F1843E910509F064C023C020910F
:10288000970220FD4FC021FD4DC008958091970211
:1028900080FD44C08091980280FF44C080919702DF
:1028A00084FD42C083EE4DC08091970282FF38C004
:1028B000F5CF8091970282FD33C08091980280FD10
:1028C00031C0ECCF8091980281FF32C08091970295
:1028D00084FD2AC087EE35C08091970283FF26C011
:1028E000F5CF8091970283FD21C08091980281FDF0
:1028F0001FC0ECCF8091970285FD1CC01DC0809148
:10290000970285FD19C016C08091970286FD16C0FA
:1029100017C08091970286FD13C010C089E311C0D3
:1029200082EE0FC080EE0DC080E00BC086EE09C0C5
:1029300084EE07C089E205C085E303C08AE201C0D6
:1029400081E390E008959091970292FF0DC0282FA7
:102950002871283019F4877F846006C0282F2471DD
:10296000243011F48B7F886093FF0DC0282F2871CD
:10297000283119F4877E846106C0282F2471243100
:1029800011F48B7E88612091980220FF0DC0382FB2
:102990003871383019F4877F816006C0382F317163
:1029A000313011F48E7F886021FF0DC0282F2871EF
:1029B000283119F4877E816106C0282F21712131C9
:1029C00011F48E7E886194FD877E089508950E949B
:1029D0006411811102C00E940C120E946F11809339
:1029E00064020E94771190939802809397020E944C
:1029F000E6140E947311682F70E080E090E00E945E
:102A0000740B609103027091040280910502909111
:102A100006020C94AC0BE82FF0E0E256FD4F8081EB
:102A20000895CF92DF92EF92FF920F931F93CF936F
:102A3000DF9389E591E00E9415058EE9E82E82E09A
:102A4000F82EC0E0D0E094E5C92E91E0D92E0CE438
:102A500011E0DF93CF93DF92CF920E94AE0581E524
:102A600091E00E941505F70181917F010E94960671
:102A70001F928F931F930F930E94AE058AE491E0FB
:102A80000E94150521968DB79EB708960FB6F8944B
:102A90009EBF0FBE8DBFC530D105D9F6DF91CF9156
:102AA0001F910F91FF90EF90DF90CF90089580EAF3
:102AB0008A95F1F7089500C008950C94571508956C
:102AC0000C945F150C9460150C945F150C946415B0
:102AD000F894E82FE295EF70F0E031A1282F2F70E5
:102AE00081E090E001C0880F2A95EAF7982F909531
:102AF000932391A392A1892B82A3789408950F9395
:102B00001F93CF93DF93CFE7D1E089918F3F11F0EF
:102B10000E94681581E0C438D807B9F7CBE7D1E047
:102B20000FE711E089918F3F11F00E9468150C1793
:102B30001D07C1F7DF91CF911F910F910895CF929B
:102B4000DF92EF92FF920F931F93CF93DF938C014D
:102B5000C62FD0E0CE0181589E4F7C01FC019081B0
:102B60009F3F09F447C0D62EF894E92FE295EF7005
:102B7000F0E081A19F7021E030E001C0220F9A9522
:102B8000EAF7822B81A382A12095282322A378949F
:102B90000E945B15EBE7F1E04FE751E031E0C12C1B
:102BA00021912F3F89F0A22FA295AF70B0E09096AF
:102BB0008C9190E02F7002C0959587952A95E2F749
:102BC00080FD02C0832F01C080E0C82A330F4E175A
:102BD0005F0731F7F70180818F3F11F00E94681580
:102BE00061E0C11001C060E08D2D0E945D15C00F35
:102BF000D11FC882DF91CF911F910F91FF90EF906D
:102C0000DF90CF9008950E947F1585E0EEE9F2E015
:102C1000DF01982F1D929A95E9F7E9E9F2E0DF01CB
:102C20001D928A95E9F785E00E945F160C940906CB
:102C3000FF920F931F93CF93DF9300D000D01F928A
:102C4000CDB7DEB78E010F5F1F4F85E0F8011192FF
:102C50008A95E9F7F12C6F2DC8010E949F15F39416
:102C6000F5E0FF12F8CF45E050E0B80189E992E0C5
:102C70000E94ED28FF24F394009709F4F12C892B8E
:102C800041F085E0F801A9E9B2E001900D928A9542
:102C9000E1F72F2D45E06EE972E089E992E00E94AC
:102CA00060160E940B068F2D0F900F900F900F90C3
:102CB0000F90DF91CF911F910F91FF90089508958C
:102CC000FF920F931F93CF93DF938C01F62ED72F94
:102CD000C42F222349F081E0809367020E94AB2039
:102CE0009093660280936502809167028823C1F009
:102CF00080916502909166020E94C320059780F042
:102D0000EF2DFD2FD8014C2F50E0CD01801B910BF2
:102D1000841795071CF48D918193F7CF1092670269
:102D2000DF91CF911F910F91FF9008950E94792319
:102D30000E9450120C9485230E9489230E94DE1267
:102D40000C94A7230E9449200E9460230E943E12F7
:102D50000E9496160E949C160E944812FBCF8091FA
:102D60006E0280FF06C06091090170E0660F771F58
:102D700026C081FF04C06091090184E005C082FF84
:102D800007C06091090188E0689FB001112417C055
:102D900090916D029923D1F060910801961788F700
:102DA0002091090188E0289F90011124929FA001A1
:102DB000939F500D112470E0CA010E94BF28603813
:102DC000710540F46115710519F406C068E070E002
:102DD000862F08958FE7089581E0089580916E020F
:102DE00080FF08C06091050170E075956795759545
:102DF000679521C081FF06C06091050170E075955F
:102E0000679519C082FF04C06091050170E010C091
:102E100090916C02992399F0609104019617A0F7A4
:102E200080910501899FC001112470E00E94BF2894
:102E30006038710540F46115710519F406C061E050
:102E400070E0862F08958FE7089581E008958D3E04
:102E500021F40E94AF16819504C08E3E29F40E9491
:102E6000AF168093720208958F3E21F40E94AF1630
:102E7000819504C0803F29F40E94AF1680937102AF
:102E80000895893F19F40E94EE1605C08A3F31F477
:102E90000E94EE1681958093730208958B3F21F472
:102EA0000E94EE16819504C08C3F29F40E94EE1614
:102EB0008093740208959FE0980F983078F421E091
:102EC00030E0A90102C0440F551F9A95E2F7CA01EC
:102ED00090917002892B8093700208958D3F21F4A8
:102EE00080916E0281600BC08E3F21F480916E0252
:102EF000826005C08F3F29F480916E0284608093C8
:102F00006E0208958D3E39F49091720297FF35C09C
:102F10001092720259C08E3E29F4909172021916D5
:102F2000BCF32BC0909171028F3E29F497FF25C00E
:102F30001092710249C0803F19F41916CCF31DC0DC
:102F400090917302893F29F41916BCF41092730210
:102F50003BC08A3F19F497FF10C0F8CF8B3F39F47C
:102F60009091740297FF09C0109274022DC08C3F9B
:102F700021F4909174021916BCF39FE0980F9830D9
:102F800080F421E030E0A90102C0440F551F9A955A
:102F9000E2F7CA01809590917002892380937002B4
:102FA00013C08D3F21F480916E028E7F0BC08E3F47
:102FB00021F480916E028D7F05C08F3F29F48091AE
:102FC0006E028B7F80936E0280917102811106C028
:102FD00080917202811102C010926D028091730281
:102FE000811106C080917402811102C010926C029E
:102FF00008958091640283FF7EC08FE891E00E9473
:103000001505809170021F928F938AE891E09F933B
:103010008F930E94AE0588E891E00E94150580918B
:103020007102282F082E000C330B3F938F9385E8F5
:1030300091E09F938F930E94AE0583E891E00E94F8
:10304000150580917202282F082E000C330B3F9338
:103050008F9380E891E09F938F930E94AE058EE757
:1030600091E00E94150580917302282F082E000C14
:10307000330B3F938F938BE791E09F938F930E9445
:10308000AE0589E791E00E94150580917402282F12
:10309000082E000C330B3F938F9386E791E09F93AC
:1030A0008F930E94AE0583E791E00E941505809101
:1030B0006D021F928F9380E791E09F938F930E9400
:1030C000AE058EE691E00E94150580916E021F927A
:1030D0008F938BE691E09F938F930E94AE0588E6D5
:1030E00091E00E9415058DB79EB74C960FB6F894E7
:1030F0009EBF0FBE8DBF0E94AB2020917102211197
:1031000004C020917202222321F090936B028093DD
:103110006A0220917302211104C0209174022223BB
:1031200021F090936902809368028FE692E00C94FC
:10313000891FEF92FF920F931F93CF93DF9300D0DD
:1031400000D000D0CDB7DEB786E0EFE6F2E0DE01DA
:10315000119601900D928A95E1F7E0907102F0903E
:103160007202009173021091740210927102109217
:1031700072021092730210927402E11003C0FF20D9
:1031800009F45DC080916A0290916B020E94C32095
:10319000AC0190916D02992339F020910A0130E041
:1031A0002417350758F04BC020910B018AE0289F67
:1031B000900111242417350718F041C09F3F19F0E2
:1031C0009F5F90936D02EE2061F00E94AF161E1477
:1031D00014F09FEF01C091E0989F902D11249093DF
:1031E0007102FF2061F00E94AF161F1414F09FEFD0
:1031F00001C091E0989F902D11249093720230911C
:1032000071023323E1F0209172022223C1F045EBD9
:103210003403C0011124992319F09093710203C063
:1032200081E08093710235EB2303C00111249923BF
:1032300019F09093720203C081E080937202011131
:1032400003C0112309F45DC0809168029091690266
:103250000E94C320AC0190916C02992339F0209117
:10326000060130E02417350758F04BC020910701C4
:103270008AE0289F900111242417350718F041C0D7
:103280009F3F19F09F5F90936C02002361F00E94B2
:10329000EE16101614F09FEF01C091E0989F902D4C
:1032A000112490937302112361F00E94EE161116FF
:1032B00014F09FEF01C091E0989F902D11249093FE
:1032C0007402309173023323E1F0209174022223BF
:1032D000C1F045EB3403C0011124992319F09093F8
:1032E000730203C081E08093730235EB2303C001B6
:1032F0001124992319F09093740203C081E0809304
:1033000074028091710281110BC08091720281114F
:1033100007C080917302811103C0809174028111F2
:103320000E94F917EB82FC820D831E8386E0FE016A
:103330003196AFE6B2E001900D928A95E1F72696BC
:103340000FB6F894DEBF0FBECDBFDF91CF911F91B6
:103350000F91FF90EF900895EFE6F2E086E0DF0135
:103360001D928A95E9F710926D0210926C021092EC
:103370006E020895CF93DF93EC01FB0182818823D5
:1033800009F43CC1C430FDE5DF0760F4CB3F9CE5A8
:10339000D90788F49E0122503C452431310508F0BC
:1033A0002EC109C0C236EDE5DE0729F0C63AFDE5BB
:1033B000DF0709F024C10E9477119093980280934F
:1033C0009702C1318CE5D80709F4C6C008F042C0A5
:1033D000C930ECE5DE0709F49BC000F5C5308CE58B
:1033E000D80709F485C078F4C330ECE5DE0709F4AA
:1033F00078C008F07AC0C230DC4509F0F5C0809191
:1034000097028160EFC0C7309CE5D90709F478C006
:1034100008F07AC0809197028061E4C0CD30FCE56D
:10342000DF0709F487C058F4CB309CE5D90709F4CD
:1034300079C008F07BC08091970288606FC0CF3060
:10344000FCE5DF0709F480C008F082C08091970294
:10345000877FC8C0CE3F9CE5D90709F471C000F54D
:10346000C531FCE5DF0709F485C068F4C3319CE58C
:10347000D90709F475C008F095C00E941C0B809113
:1034800097028F77AFC0CC3FFCE5DF07A9F108F0CA
:1034900054C0CB3FDC4509F0A7C08091980240C0E2
:1034A000C230EDE5DE0709F489C058F4C1158DE599
:1034B000D80709F45AC008F069C080919802826068
:1034C0002FC0C236EDE5DE0709F47CC0C63AFDE543
:1034D000DF0709F481C0C330DD4509F085C080E015
:1034E0006EC08091970282607DC08091970216C065
:1034F00080919702886076C08091980282604FC068
:103500008091970280626EC08091970280646AC049
:103510000E941C0B80919702806864C0846062C026
:1035200081603DC0809197028E7F5CC08091970240
:103530008D7F58C08091970216C08091980218C064
:10354000809198028D7F2BC0809197028F7E4AC018
:10355000809197028F7D46C0809197028F7B42C0F9
:1035600080919702877F8B7F3DC0809198028D7FED
:103570008E7F15C08091970282FB222720F991E06F
:10358000922790FB82F990FB83F92CC080919802DE
:10359000982F909591708E7F892B90FB81F9809365
:1035A000980222C00E941C0B8091970287FB222761
:1035B00020F991E0922790FB87F914C081E00E94E6
:1035C0000E1212C08091970284FB222720F991E00D
:1035D000922790FB84F906C080919702982F9095CE
:1035E00090FB80F9809397028091970290919802C6
:1035F0000E9488110E941C0B80E001C081E0DF91D5
:10360000CF910895809104011F928F9380910501BD
:103610001F928F93809108011F928F9380910901CF
:103620001F928F9380910A011F928F9380910B01BB
:103630001F928F9382EB91E09F938F930E94AE0530
:103640008DB79EB70E960FB6F8949EBF0FBE8DBF76
:103650000895883220F58E3108F068C08B3091F1E2
:10366000C0F4873009F0BEC081E080930B0184E193
:1036700080930A018AE0809309018EE1809308011A
:1036800088E08093050188E28093040184E193E05F
:10369000C6C0833109F443C0843169F1A3C08F34BB
:1036A00009F49EC028F4893231F1883359F09AC068
:1036B000813531F008F4D4C0823509F4A7C092C036
:1036C0008FEFA5C086E393E00E9415050E94021BC0
:1036D0001F9281E08F931F9288E08F938FE292E098
:1036E0009F938F930E94AE050F900F900F900F90B5
:1036F0000F900F9096C083E393E00E941505809190
:103700007902882309F4AAC01092790210927802F3
:10371000109277021092760210927502B1C085E283
:1037200093E00E9415050E94021B7BC08D5180937F
:103730007902833031F170F48130D1F0823009F0B8
:103740003FC08AE091E0909378028093770281E90C
:1037500091E01FC0853059F108F1863089F584E089
:1037600091E090937802809377028CEC91E011C005
:103770008BE091E0909378028093770288E891E063
:1037800008C089E091E090937802809377028DE9F8
:1037900091E0909376028093750218C088E091E0E2
:1037A00090937802809377028AEA91E0F2CF85E0E5
:1037B00091E0909378028093770289EB91E0E9CFD2
:1037C0001092790282E293E00E94150580917902BD
:1037D000882309F455C01F928F938EE193E00DC0AA
:1037E0008AE015C081E193E01AC097FF47C01082BC
:1037F00080811F928F938BE093E09F938F930E9421
:10380000AE050F900F900F900F900BC081E0E091EC
:103810007702F0917802309729F588E093E00E94D2
:10382000150520917902222359F18091750290911A
:103830007602009711F484E891E09F938F931F9292
:103840002F938FEF92E09F938F930E94AE050F907E
:103850000F900F900F900F900F9016C080E008957A
:1038600086EFD5CF2081082E000C990B820F911D79
:103870008F3F910509F00CF4B8CF8FEF8083B8CF5C
:103880008BEF92E00E94150581E00895CF93C82F39
:103890001F928F938CE493E09F938F930E94AE05C9
:1038A00081E090E0A0E0B0E0BC01CD0104C0660F73
:1038B000771F881F991FCA95D2F70E94740B0F902B
:1038C0000F900F900F90CF910C941C0BEF92FF92E2
:1038D0000F931F93CF93DF938B3109F4EDC008F062
:1038E0008EC08B3009F4B1C008F078C0863009F47E
:1038F000AFC020F4853009F4BDC04EC1873009F453
:10390000C0C0883009F048C10E9473111F928F9384
:103910008FE697E09F938F930E94AE050E946F11F0
:1039200083FB992790F91F929F9382FB992790F927
:103930001F929F9381FB992790F91F929F93982F35
:1039400091701F929F931F928F9386E297E09F93AF
:103950008F930E94AE050E94771187FB222720F9E2
:103960001F922F9386FB222720F91F922F9385FB0E
:10397000222720F91F922F9384FB222720F91F92E0
:103980002F9383FB222720F91F922F9382FB22275C
:1039900020F91F922F9391FB222720F91F922F933A
:1039A000292F21701F922F9381FB222720F91F922C
:1039B0002F93282F21701F922F939F938F9381E431
:1039C00096E09F938F930E94AE058DB79EB7889621
:1039D0000FB6F8949EBF0FBE8DBF35C0803109F47D
:1039E00095C020F48E3009F47BC0D6C0863109F42E
:1039F000A8C0893109F0D0C08CEB93E084C08A3232
:103A0000E1F060F4873209F4C3C028F48E3108F481
:103A1000C3C08D51BEC0893269F1BEC0833448F441
:103A20008A3308F0B3C0853309F4B2C0883369F033
:103A3000B3C0833409F4ACC0AFC08AE198E00E94FF
:103A400015050E940C12C1E0ACC08EE994E05BC089
:103A500080916402817F8E7F8093640287E794E087
:103A60000E94150586E198E00E94150581E080938B
:103A70007A02E9CF8AEF97E00E9415050E940E06B0
:103A8000E2CF80916402C82FC095C170C0FB80F95D
:103A900080936402CC2329F08EEE97E00E941505F6
:103AA00080C081EE97E00E94150580916402897FB5
:103AB000877F80936402C7CF9091640291FBCC27EB
:103AC000C0F981E0C827892FC0FB81F98093640287
:103AD000CC2319F084ED97E029C086EC97E013C061
:103AE0009091640292FBCC27C0F981E0C827892F0E
:103AF000C0FB82F980936402CC2319F087EB97E036
:103B000015C087EA97E00E9415059DCF9091640249
:103B100093FBCC27C0F981E0C827892FC0FB83F92C
:103B200080936402CC2351F08BE997E00E94150545
:103B30008091640281608093640233C08EE897E0D4
:103B4000E2CF0E94B720162F072FF82EE92ED09132
:103B50009602C09118010E94341FEF92FF920F93BA
:103B60001F931F92DF931F92CF931F928F9381E534
:103B700093E09F938F930E94AE058DB79EB70C96EE
:103B80000FB6F8949EBF0FBE8DBF5DCF895301C0A5
:103B900080E00E94461C57CF8CE897E00E941505F4
:103BA000C0E08C2FDF91CF911F910F91FF90EF908C
:103BB000089580E008950C94D91DCF93C82F80916B
:103BC0007A02813071F040F0823009F045C08C2FCC
:103BD0000E94291B81E046C00E946D108232F1F5DF
:103BE00004C00E946D10823261F48C2F0E94DB1D94
:103BF000811104C08C2F0E94661C2CC081E090E0D3
:103C000029C08C2F0E94D91D811123C0C431C9F055
:103C100058F4CB3069F0C031B9F482E080937A0275
:103C200088E30E94291B15C0C93259F0C83361F4DA
:103C300087E794E00E94150588E493E00E9415054B
:103C400008C010927A020CC086E493E00E94150529
:103C500007C081E0817006C010927A0280E002C045
:103C600080E0F8CFCF910895CF93DF9386319C45C4
:103C700041F5EB010E946D10982F8A81209102017D
:103C800030910301882379F09A7A81E009F480E089
:103C900080937B02911102C069E201C065E3C90112
:103CA0000E9405200AC080917B02811102C069E256
:103CB00001C065E3C9010E9407200E94AF1080E0A7
:103CC00001C081E0DF91CF9108950F931F93CF93AF
:103CD000DF93C42FD22FFC0182818823C9F0409347
:103CE0007E020E94AB2090937D0280937C0280E252
:103CF0008C0F883008F057C0C77081E001C0880F72
:103D0000CA95EAF7DF91CF911F910F910C94790832
:103D100080917E02481330C080917C0290917D0298
:103D20000E94C320883C910538F510E21D0FCD1785
:103D3000B9F080E28C0F883040F4C77081E001C098
:103D4000880FCA95EAF70E948008183028F581E0AC
:103D50009D2F977001C0880F9A95EAF70E94790805
:103D6000802F0E9470081830F0F4D77081E001C0F5
:103D7000880FDA95EAF70AC080E28C0F883098F451
:103D8000C77081E001C0880FCA95EAF7DF91CF9133
:103D90001F910F910C948008802FDF91CF911F917C
:103DA0000F910C947008DF91CF911F910F9108959E
:103DB0000F939C01CB01243F4CE5340731F188F48B
:103DC000293DFCE53F07D9F02A3D4CE5340779F160
:103DD000283D3C45A9F506E221EE41EE68ED7CE583
:103DE0002BC0263FFCE53F07E1F0A8F0273F3C450C
:103DF00039F507E225EE46EE67EF7CE51DC007E2E8
:103E000025EE45EE69ED7CE517C006E221EE40EEB9
:103E100064EF7CE511C007E225EE44EE65EF7CE53A
:103E20000BC006E221EE42EE66EF7CE505C008E23B
:103E300021E045EE6AED7CE50E94651E80E008C049
:103E4000FC018281882319F010927E0201C081E07A
:103E50000F9108959093F1018093F001089590934C
:103E60008402809383020895E0918302F09184029A
:103E7000309721F00190F081E02D099480E00895C1
:103E8000EF92FF920F931F93CF93DF93E091830202
:103E9000F09184023097B1F18C010280F381E02D22
:103EA00009958091640282FF2DC080FF04C083E3E6
:103EB00098E00E941505E80118E08DE2E82E88E000
:103EC000F82E8091640280FF0BC088811F928F932F
:103ED000FF92EF920E94AE050F900F900F900F90FF
:103EE000115021961111EDCF8091640280FF0AC01C
:103EF0008BE298E0DF91CF911F910F91FF90EF90AF
:103F00000C941505DF91CF911F910F91FF90EF90C9
:103F10000895E0918302F0918402309739F022E015
:103F2000DC012C930480F581E02D09940895209103
:103F30008102309182022817390771F09093820232
:103F400080938102E0918302F0918402309721F006
:103F50000680F781E02D0994089520917F02309129
:103F600080022817390771F09093800280937F02B6
:103F7000E0918302F0918402309721F00084F18572
:103F8000E02D09940895FC01329697E080E091506D
:103F900029F021912223D9F38F5FF9CF0895662369
:103FA00049F0FC01329608962191621729F0E81732
:103FB000F907D1F780E0089581E008959C01FC01A4
:103FC00032969FEF80E04191461789F09F3F19F4A8
:103FD000411101C0982F8F5F8630A9F79F3F39F0BC
:103FE000F901E90FF11D97FDFA956283089508958F
:103FF0009C012A5F3F4FFC014281461301C012829F
:10400000019682179307B9F708950C94DE1F0C945C
:10401000F81F029626E0FC0111922A95E9F708950F
:1040200008950C94102083E0809385020C94112055
:10403000811102C081E001C082E0809385020C946E
:1040400011200C94182081E0809385020C9411209B
:104050000C94232008950C942A200C942B200C946B
:104060002A200C942A200C942A20CF930E943120DD
:104070000E9418160E942F20C0E08C2F0E940B1562
:10408000811104C0CF5FC530C1F701C081E0CF917D
:10409000089508951F920F920FB60F9211248F93D7
:1040A0009F93AF93BF9380918602811113C080913B
:1040B000A3029091A402A091A502B091A6024196FC
:1040C000A11DB11D8093A3029093A402A093A50209
:1040D000B093A602BF91AF919F918F910F900FBEA9
:1040E0000F901F9018958091AB02843031F10E949F
:1040F0008E061092860220E488E190E00FB6F894D4
:10410000A895809360000FBE2093600083B7817FE5
:10411000846083BF83B7816083BF7894889583B7B9
:104120008E7F83BF0FB6F894A89580916000886158
:1041300080936000109260000FBE08950E941C0BD7
:104140000C94920682E084BD93E095BD9AEF97BDF2
:1041500080936E0008952FB7F8948091A3029091F8
:10416000A402A091A502B091A6022FBF08952FB777
:10417000F8946091A3027091A4028091A50290919D
:10418000A6022FBF08959C014FB7F8948091A30217
:104190009091A402A091A502B091A6024FBF821BEC
:1041A000930B089578941F920F920FB60F921124DB
:1041B0008F939F93AF93BF938091A3029091A4029A
:1041C000A091A502B091A6020196A11DB11D8093F8
:1041D000A3029093A402A093A502B093A602BF915C
:1041E000AF919F918F910F900FBE0F901F901895D8
:1041F000F89481E08093E00080E28093D800E9ECBD
:10420000F0E010828FE19EE40197F1F700C000001A
:104210001DBA109268001CBC10BE1FBA10927A0022
:1042200010926E0010926F00109271001092720046
:104230001082ECEBF0E0108214B817B81AB81DB871
:1042400010BA108215B818B81BB81EB811BA0C9461
:10425000003F0895809195020895089522E02093EB
:10426000E9002FEF3091E800215035FD06C035ED13
:104270003A95F1F700002111F5CF2091E80025FFD4
:104280000BC040E050E066E070E00E941624809190
:10429000E8008E778093E8000895CF93DF9321E0C4
:1042A0002093E9002FEF3091E800215035FD06C042
:1042B00035ED3A95F1F700002111F5CF2091E80096
:1042C00025FF14C0EC0140E050E068E070E00E947F
:1042D00016248091E8008E778093E80088E0FE0144
:1042E000ADE8B2E001900D928A95E1F7DF91CF91B0
:1042F00008958093890270938B0260938A02809163
:10430000AB02843001F582E08093E9008FEF909159
:10431000E800815095FD06C095ED9A95F1F70000F3
:104320008111F5CF8091E80085FF0DC040E050E09D
:1043300063E070E089E892E00E9416248091E80032
:104340008E778093E8000895BC0184E00C94792175
:10435000BC0183E00C94792189E598E00E94150561
:104360008091AA02811109C00E94A7250E940426FB
:104370008091E20084608093E200089585E598E0F2
:104380000E9415051092AA02089581E598E00E9406
:1043900015050C9428208DE498E00E941505609185
:1043A000A70281E0611101C080E00C94132089E430
:1043B00098E00E9415059091AB0281E0943009F0DD
:1043C00080E06091A7020C941820209188022F5F52
:1043D000822F62E30E94B328992319F02093880268
:1043E00008951092880280918C02882371F1809147
:1043F000AB02843041F58091E9008F702091EC0090
:10440000922F917020FD90E8892B93E09093E90022
:104410009091EB0090FF14C09091EE0097FF10C0B8
:104420009091E80095FF03C01092F100F9CF9091B0
:10443000E80090FF05C09091E8009E779093E80017
:104440008F708093E90010928C02089542E061EC35
:1044500081E00E94202542E261EC82E00E9420255A
:1044600042E261EC83E00E9420259091AB0281E062
:10447000943009F080E06091A7020C942120809193
:10448000AD02833009F461C030F4813071F08230C4
:1044900009F49AC008958A3009F486C08B3009F473
:1044A0006CC0893009F0A8C020C08091AC02813A6C
:1044B00009F0A2C08091E800877F8093E800809196
:1044C000B0029091B102892B21F468E08DE892E06E
:1044D00003C060E080E090E070E00E946124809181
:1044E000E8008B778093E80008958091AC028132D8
:1044F00009F082C08091B0029091B102029708F059
:104500007BC08091E800877F8093E8008091E8007D
:1045100082FD05C08091AB028111F8CF6DC0209162
:10452000F3008091F20090E0922B029731F4809199
:10453000F100813011F0863021F48091F1008093F8
:1045400095028091E8008B7753C08091AC02813A4C
:1045500009F052C08091B0029091B102892B09F00C
:104560004BC08091E800877F8093E8008091E8004D
:1045700080FFFCCF8091180136C08091AC0281325F
:10458000D9F58091B0029091B102892BA9F5809163
:10459000E800877F8093E8000E9455258091AE0255
:1045A000809318010C941C0B8091AC02813221F590
:1045B0008091E800877F8093E8000E9455258091D4
:1045C000AF028093960208958091AC02813AA1F4E3
:1045D0008091E800877F8093E8008091E80080FF69
:1045E000FCCF809196028093F1008091E8008E7755
:1045F0008093E8000C94552508959FB7F894109285
:104600008C029FBF9091AB02943009F057C09091FB
:10461000E9009F703091EC00232F217030FD20E8DD
:10462000922B23E02093E9002091EB0020FF43C070
:104630002091EE0027FF3FC020918702222321F026
:104640002091E80025FF37C01092870226E03091C4
:10465000E80035FD15C03091AB02343061F5309182
:10466000EB0035FD28C0215021F481E080938702C2
:1046700022C0EFE9FFE03197F1F700C00000E7CF7B
:104680008093F1008091E80085FD0AC08091E800E8
:1046900080FFFCCF8091E8008E778093E80006C011
:1046A0008FB7F89421E020938C028FBF9F70909376
:1046B000E90080E008959F709093E9008FEF0895DE
:1046C00084B7877F84BF0FB6F894A8958091600067
:1046D000886180936000109260000FBE90E080E8D7
:1046E0000FB6F89480936100909361000FBE0C9414
:1046F00023200E94A7250E940426E2EEF0E080819C
:104700008460808378940C9498288CE091E00C94D9
:104710002F1F8091AB028530C9F485E498E00E9498
:1047200015058091AB02853079F40E947320809149
:10473000A9028823B1F30E943520882391F30E94B7
:1047400000240E941C0BEDCF0C949E200895089528
:104750000C94AA23292F332723303105C9F060F4A4
:104760002130310581F02230310509F041C08BE55F
:1047700090E029E838E040C021323105E1F02232F2
:10478000310531F135C082E190E024EE38E034C0EB
:1047900099278130910549F028F0029749F5EDE518
:1047A000F8E005C0E5E8F8E002C0E3E7F8E084914E
:1047B00090E09F0121C063307105D0F4660F771F30
:1047C000FB01E651FE4F2081318189E090E014C069
:1047D0006330710568F4FB01EE0FFF1FEC51FE4FD3
:1047E00020813181FB01EF51FE4F808190E004C0B8
:1047F00080E090E020E030E0FA01318320830895EA
:1048000080E189BD82E189BD09B400FEFDCF8091C0
:10481000D8008F7D8093D8008091E00082608093E3
:10482000E0008091E00081FDFCCF0895CF92DF92FF
:10483000EF92FF920F931F93CF93DF93EC018B01C5
:104840007A010E947425811133C0E114F10439F01A
:10485000F70180819181081B190BC80FD91FC12C4A
:10486000D12C0115110519F18091E80085FD16C0C4
:104870008091E8008E778093E800E114F10449F01C
:10488000F70180819181C80ED91ED182C08285E056
:104890000FC00E947425882321F30AC08991809358
:1048A000F10001501109FFEFCF1ADF0ADACF80E0E3
:1048B000DF91CF911F910F91FF90EF90DF90CF90FC
:1048C00008952091B2023091B3022617370748F0BD
:1048D0006115710539F42091E8002E772093E800E6
:1048E00001C0B901FC0120E06115710579F18091E9
:1048F000AB028823F1F18530F1F18091E80083FD6E
:104900003CC08091E80082FD2EC08091E80080FFCD
:10491000EBCF2091F3008091F20090E0922B611593
:10492000710551F08830910538F421912093F10000
:10493000615071090196F3CF21E0089709F020E05A
:104940008091E8008E778093E800CECF2111CFCF01
:104950000AC08091AB02882361F0853061F08091BC
:10496000E80083FD0AC08091E80082FFF2CF80E07A
:10497000089582E0089583E0089581E008952091EC
:10498000B2023091B3022617370748F0611571055E
:1049900039F42091E8002E772093E80001C0B90196
:1049A000FC0120E06115710591F18091AB02882333
:1049B00009F440C0853009F43FC08091E80083FDD0
:1049C0003DC08091E80082FD2FC08091E80080FF0B
:1049D000E9CF2091F3008091F20090E0922B6115D5
:1049E000710559F08830910540F424912093F1002D
:1049F0003196615071090196F2CF21E0089709F0D4
:104A000020E08091E8008E778093E800CBCF2111E1
:104A1000CCCF0AC08091AB02882361F0853061F071
:104A20008091E80083FD0AC08091E80082FFF2CF08
:104A300080E0089582E0089583E0089581E008957C
:104A4000982F973068F59093E900981739F0709196
:104A5000EC002091ED005091F00003C0242F762F40
:104A600050E021FD02C09F5FECCF3091EB003E7F14
:104A70003093EB003091ED003D7F3093ED003091AD
:104A8000EB0031603093EB007093EC002093ED006D
:104A90005093F0002091EE0027FDE5CF80E00895CF
:104AA0008F708093E90081E008958091AC0287FFC8
:104AB00011C08091E80082FD05C08091AB02811198
:104AC000F8CF11C08091E8008B770BC08091AB02CA
:104AD000882349F08091E80080FFF8CF8091E800BA
:104AE0008E778093E80008952091E4003091E500EE
:104AF00095E64091EC00842F817040FF23C08091A7
:104B0000E80080FD1DC08091AB02882399F08530BC
:104B100099F08091EB0085FD11C04091E400509127
:104B2000E5002417350729F3915011F09A01E1CFE0
:104B300084E0089582E0089583E0089581E0089577
:104B400080E008954091E80042FFDDCF08950E9483
:104B500015260E941D26E0EEF0E0808181608083B2
:104B6000E8EDF0E080818F77808319BCA7EDB0E09D
:104B70008C918E7F8C9380818F7E80831092AA028D
:104B800008950F931F93CF93DF930E9415260E94E1
:104B90001D26C8EDD0E088818F7788838881806862
:104BA000888388818F7D888319BC1092AB02109214
:104BB000A7021092A9021092A80200EE10E0F801DC
:104BC00080818B7F808388818160888342E060E080
:104BD00080E00E942025E1EEF0E080818E7F8083DE
:104BE000E2EEF0E080818160808380818860808354
:104BF000F80180818E7F8083888180618883DF9146
:104C0000CF911F910F910895E8EDF0E080818F7EA4
:104C10008083E7EDF0E080818160808384E082BF63
:104C200081E08093AA020C94C125E8EDF0E0808138
:104C30008E7F80831092E20008951092DA00109225
:104C4000E10008951F920F920FB60F9211242F9337
:104C50003F934F935F936F937F938F939F93AF9304
:104C6000BF93EF93FF938091E10082FF0BC080918F
:104C7000E20082FF07C08091E1008B7F8093E1001A
:104C80000E94E5218091DA0080FF1FC08091D8004A
:104C900080FF1BC08091DA008E7F8093DA008091C4
:104CA000D90080FF0DC080E189BD82E189BD09B4D2
:104CB00000FEFDCF81E08093AB020E94AC2105C0D5
:104CC00019BC1092AB020E94BE218091E10080FFCE
:104CD00019C08091E20080FF15C08091E2008E7FB4
:104CE0008093E2008091E20080618093E2008091F5
:104CF000D80080628093D80019BC85E08093AB0215
:104D00000E94CB218091E10084FF30C08091E200BD
:104D100084FF2CC080E189BD82E189BD09B400FE19
:104D2000FDCF8091D8008F7D8093D8008091E100E5
:104D30008F7E8093E1008091E2008F7E8093E2007D
:104D40008091E20081608093E2008091A702882335
:104D500011F084E007C08091E30087FD02C081E08C
:104D600001C083E08093AB020E94D7218091E100D3
:104D700083FF29C08091E20083FF25C08091E1007C
:104D8000877F8093E10082E08093AB021092A702BC
:104D90008091E1008E7F8093E1008091E2008E7F20
:104DA0008093E2008091E20080618093E20042E023
:104DB00060E080E00E9420258091F0008860809370
:104DC000F0000E94C521FF91EF91BF91AF919F919B
:104DD0008F917F916F915F914F913F912F910F90A4
:104DE0000FBE0F901F9018951F920F920FB60F9243
:104DF00011242F933F934F935F936F937F938F93E0
:104E00009F93AF93BF93CF93DF93EF93FF93C091A3
:104E1000E900CF708091EC00D82FD17080FDD0E8F0
:104E20001092E9008091F000877F8093F0007894E1
:104E30000E9438271092E9008091F00088608093EA
:104E4000F000CD2BCF70C093E900FF91EF91DF917F
:104E5000CF91BF91AF919F918F917F916F915F9112
:104E60004F913F912F910F900FBE0F901F9018956B
:104E70001F93CF93DF93CDB7DEB7AA970FB6F89401
:104E8000DEBF0FBECDBFECEAF2E08091F10081936E
:104E900022E0E43BF207C9F70E943F228091E8003C
:104EA00083FF2EC18091AC029091AD02492F50E05A
:104EB0004A30510508F024C1FA01EE59FF4F0C9415
:104EC000D328803821F0823809F01AC108C08091B7
:104ED000A8029091A902992389F082600FC0809165
:104EE000B0028F70873008F00BC18093E900809189
:104EF000EB0085FB882780F91092E9009091E8008B
:104F0000977F9093E8008093F1001092F100D1C058
:104F1000282F2D7F09F0F4C0882319F0823061F02A
:104F2000EFC08091AE02813009F0EAC0933009F001
:104F300080E08093A9022EC08091AE0281112AC028
:104F40008091B0028F702FEF280F263008F0D8C064
:104F50008093E9002091EB0020FF1CC0933021F4E6
:104F60008091EB00806214C09091EB00906190936F
:104F7000EB0021E030E0A90102C0440F551F8A95E3
:104F8000E2F74093EA001092EA008091EB0088601B
:104F90008093EB001092E9008091E800877F809376
:104FA000E8000E945525ACC08111AAC01091AE0244
:104FB0001F778091E3008078812B8093E3008091BC
:104FC000E800877F8093E8000E9455258091E800E3
:104FD00080FFFCCF8091E30080688093E300111193
:104FE00002C082E001C083E08093AB0289C0805898
:104FF000823008F085C08091AE029091AF028C3D66
:1050000053E0950779F583E08A838AE289834FB775
:10501000F894DE01139620E03EE051E2E32FF0E049
:1050200050935700E49120FF03C0E295EF703F5F7B
:10503000EF708E2F90E0EA3010F0C79601C0C09656
:105040008D939D932F5F243149F74FBF8091E800E6
:10505000877F8093E8006AE270E0CE0101960E94AB
:10506000612416C06091B0027091B102AE014F5F31
:105070005F4F0E94A823BC01892B09F441C0909185
:10508000E800977F9093E80089819A810E94BF246D
:105090008091E8008B778093E80032C0803881F5FA
:1050A0008091E800877F8093E8008091A702809339
:1050B000F1008091E8008E7772CF811121C080913C
:1050C000AE029091AF0299270297D4F48091E80044
:1050D000877F8093E8008091AE028093A7020E94B0
:1050E00055258091A702811106C08091E30087FDBC
:1050F00002C081E001C084E08093AB020E942622BE
:105100008091E80083FF0AC08091E800877F809348
:10511000E8008091EB0080628093EB00AA960FB6C6
:10512000F894DEBF0FBECDBFDF91CF911F910895E0
:10513000CF938091AB028823A1F0C091E900CF709A
:105140009091EC00892F817090FD80E8C82B10921F
:10515000E9008091E80083FD0E943827CF70C0935A
:10516000E900CF910895991B79E004C0991F961723
:1051700008F0961B881F7A95C9F78095089597FBCC
:10518000072E16F4009407D077FD09D00E94D92885
:1051900007FC05D03EF4909581959F4F089570953A
:1051A00061957F4F0895EE0FFF1F0590F491E02D5C
:1051B0000994AA1BBB1B51E107C0AA1FBB1FA6175E
:1051C000B70710F0A61BB70B881F991F5A95A9F7B0
:1051D00080959095BC01CD010895FB01DC0104C0D0
:1051E0008D910190801921F441505040C8F7881BDF
:1051F000990B0895F999FECF92BD81BDF89A992730
:1052000080B50895A8E1B0E042E050E00C942E296A
:10521000262FF999FECF92BD81BDF89A019700B46F
:10522000021639F01FBA20BD0FB6F894FA9AF99A0F
:105230000FBE08950396272F0E9409290E9408296E
:10524000252F0E940929242F0C9409290196272F24
:105250000E9409290C940829DC01CB01FC01F99971
:10526000FECF06C0F2BDE1BDF89A319600B40D92B2
:0C52700041505040B8F70895F894FFCF6B
:10527C00C8004D02280850011E0A14012A214D2194
:10528C002E21A821A4212D2101E200E900EA00B57C
:10529C0000B600B700CD008301CC008A01920194C6
:1052AC00012102230224022502260227022A02B32C
:1052BC0000B4006F007000818283E200E900EA0014
:1052CC00B500B600B700CD008301CC008A01920175
:1052DC0094012102230224022502260227022A021B
:1052EC00B300B4006F0070008182839190F5F4F6E6
:1052FC00313336353F3F3F006D6B5F64656C6179D0
:10530C00006D6B5F696E74657276616C006D6B5FBE
:10531C006D61785F7370656564006D6B5F74696D4A
:10532C00655F746F5F6D6178006D6B5F7768656545
:10533C006C5F6D61785F7370656564006D6B5F7732
:10534C006865656C5F74696D655F746F5F6D6178BE
:10535C0000407B2293091809F6089B08B408CD0875
:00000001FF
